:10000000E428A901AB01AA0006300628A6002B08A7
:100010002902031D0D282A08280204300318013084
:10002000031902302605031D0130DF282016201E8B
:100030002012A01A1F28A016552003184A282011A4
:100040000830AB006620AA0DAB0B222820192F2800
:10005000201A2B287B2075207120201A4A20782016
:1000600003102A0851282016201E2012201B3D288C
:10007000FE39A600201703105128A01B4528AE000A
:10008000A017552003184A282E08592003184A287B
:10009000201E51287B2075202013A013A0122011B0
:1000A00078203014031C3010DF286E202608A01A98
:1000B0000138AA000830AB00AA0D78200318612887
:1000C0007B2075207120AB0B5C2878207520682878
:1000D00064000310051803147120080078207520AF
:1000E0007B208510831685107E28831685147E2834
:1000F000831605147E280510831605108312080048
:10010000A200280829040319DF28D120AB01AC0183
:10011000220984178005841300008E282A08AB0763
:1001200000082204031C22068000AC0A0319A80A56
:100130000319A90F8C28220884178004DF28AD0139
:10014000AC011030AE00290DAC0DAD0D2A08AC028B
:100150002B08031C2B0FAD020318B5282A08AC0787
:100160002B0803182B0FAD070310A80DA90DAE0B1C
:10017000A3282808DF281030B200A901A801AF0C7D
:10018000AE0C031CC9282A08A8072B0803182B0F3C
:10019000A907A90CA80CAD0CAC0CB20BBF282C08FD
:1001A000DF28A809A909A80A0319A90A0800031049
:1001B000A90CA80CFF3E0318D7282808DF288313B2
:1001C0008312031300000800A00183168113073077
:1001D00083129F00043083168500E0308600823051
:1001E00092003C30831295000C309700043092004E
:1001F000EE30CB002430CC00BA30CD00B630CE008B
:100200007430CF00D630D000DE30D100A430D20020
:10021000FE30D300F630D400EF30D5002530D600C4
:10022000BB30D700B730D8007530D900D730DA00EE
:10023000DF30DB00A530DC00FF30DD00F730DE0012
:100240001030DF000130E000E101E3010230E200A4
:10025000E5010430E400E7014030E600E9018030C8
:10026000E800EB010830EA000130ED00EC01EF019D
:100270002030EE000230F100F001F3011030F20006
:10028000C7019E303520AC30352045303320212247
:100290009922861A4C29DF22061B4F294623861BEA
:1002A0005229DF2205195529DF22572147294708FE
:1002B000743E84000008C8000611831606118312DC
:1002C0008610831686100A308312C0000310470D73
:1002D000623E84000008C100840A0008C2000612C1
:1002E0008316061283124208A9004108A8004003A1
:1002F000A200A20AA90CA80CA20B7A290130031CA7
:100300000301013903190610031D0614061683168E
:1003100006128312C003400803198F29662908308A
:10032000C00048084B3E84000008C201C10006120C
:100330008316061283124208A9004108A800400350
:10034000A200A20AA90CA80CA20BA2290130031C2E
:100350000301013903190610031D0614061683163E
:1003600006128312C00340080319B7299129061207
:1003700083160612831206100616831606128312BF
:100380000615831606118312DC2308009E303520E3
:10039000C03035204A083520490833200800B40110
:1003A0004908B300F030B3050030B4053408A900A3
:1003B0003308A8000430DA20B3002908B400340858
:1003C000AF003308AE00AB010A30AA00BB20B30077
:1003D0002D08B400B6014908B5000F30B50500304E
:1003E000B60533083507C90008004308C900B40141
:1003F0004908B3003408A9003308A800AB010A304B
:10040000AA009F20B3002908B4000430A8000310FC
:10041000B30DB40DA80B072AB6014908B50036087C
:10042000A9003508A800AB010A30AA009F202D08BA
:10043000B6002C08B50033083507C900C6218F2245
:1004400008009E303520C0303520030133209F3016
:1004500035201820B8001820B9001820BA0018203C
:10046000BB001820BC001820BD001620BE003E08AE
:10047000C900CF214908BE003D08C900CF21490865
:10048000BD003C08C900CF214908BC003A08C9009A
:10049000CF214908BA003908C900CF214908B9005D
:1004A0003808C900CF214908B80007303B020319BA
:1004B0000130031D0301B70019303C02030103188A
:1004C00001303705B7003C08A8001F300120370570
:1004D00003198E2A02303A0203190130031D030169
:1004E000B700390803190130031D03013705B700B0
:1004F000380803190130031D0301370503198E2A3B
:1005000003303D02031D872A0130C900C6210A308D
:100510003D02031D8E2A0330C900C62108007F302A
:10052000AA00A9018230A80005308400083080208C
:1005300008001630F400A9013A08A800AB010A30FF
:10054000AA009F20A7002708F500A9013A08A800E3
:10055000AB010A30AA009F202C08A7002708F6004C
:100560001430F700A9013908A800AB010A30AA002D
:100570009F20A7002708F800A9013908A800AB01AF
:100580000A30AA009F202C08A7002708F900143081
:10059000FA00A9013808A800AB010A30AA009F2080
:1005A000A7002708FB00A9013808A800AB010A3002
:1005B000AA009F202C08A7002708FC00080016307E
:1005C000F4000230F500F601A9013E08A800AB01D5
:1005D0000A30AA009F20A7002708F700A9013E08BB
:1005E000A800AB010A30AA009F202D08B4002C08F7
:1005F000B3000A303307A7002708F800A9013D0817
:10060000A800AB010A30AA009F20A7002708F90024
:10061000A9013D08A800AB010A30AA009F202D08BF
:10062000B4002C08B3000A303307A7002708FA00EB
:10063000A9013C08A800AB010A30AA009F20A7002E
:100640002708FB00A9013C08A800AB010A30AA005A
:100650009F202D08B4002C08B3000A303307A700F0
:100660002708FC0008001630F4001630F50016309C
:10067000F6001630F7001630F8001630F900163084
:10068000FA001630FB003B08FC0008000130BF00F8
:100690008F2201304602031D4E2B99220230460262
:1006A000031D532BDF2203304602031D582B332337
:1006B0001530F400212278235721861A652B430830
:1006C00044020318642BC303F521861B6D2B4508D8
:1006D000430203186C2BC30AF521061B762B8F22CD
:1006E000BF0A08303F02031D762B4729DC23492B24
:1006F00001303F02031D862B0230CA003A08C300B6
:10070000C4011730C5000130C600DB2B02303F02A8
:10071000031D942B0130CA003908C300C4013B30CB
:10072000C5000130C600DB2B03303F02031DA12BA7
:10073000CA013808C300C4013B30C5000130C600FF
:10074000DB2B04303F02031DAF2B0630CA003E08EE
:10075000C300C4016330C5000230C600DB2B053086
:100760003F02031DBE2B0530CA003D08C300013007
:10077000C4000C30C5000230C600DB2B06303F023F
:10078000031DCD2B0430CA003C08C3000130C40057
:100790001F30C5000230C600DB2B07303F02031DAF
:1007A000DB2B0330CA003B08C3000130C400073014
:1007B000C5000330C6000800C70A09304702031C01
:0607C000E22BC701080056
:02400E00623F0F
:00000001FF
